:100000000C94B5050C948E1B0C94B51B0C94D20566
:100010000C94D2050C94D2050C9473090C94D2055F
:100020000C94D2050C94D2050C94D2050C94D205F4
:100030000C94D2050C94341B0C94D2050C94D2056C
:100040000C94DC1B0C94D2050C94D2050C94D205B4
:100050000C94D2050C94D2050C94D2050C94D205C4
:100060000C94D2050C94D2053008320835083708B4
:10007000390849083B083D083F084108430845083E
:10008000470849084B084D084F08510853085508C0
:10009000570859085B085D08AF08B108B808BA08E6
:1000A000BE08C008C208C408C608C808CA08DB08D9
:1000B000D308D508D708CC084516221625162816C9
:1000C0002B162E163116341637163A166916631685
:1000D000451648164B164E165116541657165A16F4
:1000E0005D1660166916631607634236B79BD8A77C
:1000F0001A39685618AEBAAB558C1D3CB7CC57634D
:10010000BD6DEDFD753EF6177231BF000000803FFA
:1001100008000000BE922449123EABAAAA2ABECD16
:10012000CCCC4C3E00000080BEABAAAAAA3E000088
:100130000000BF000000803F000000000008417880
:10014000D3BB4387D1133D190E3CC3BD4282AD2BB7
:100150003E68EC8276BED98FE1A93E4C80EFFFBEAF
:1001600001C4FF7F3F00000000000AC82E8C01D1AF
:100170008595348BAA7456BDCAE8A6CA29CB2A92A3
:10018000EECAA4362B2FAA3C439AACBC78F3D068B5
:10019000D4B26A454A2AA6C993C42909C7248DB195
:1001A000D3CD0821708A5215AA01E08063C2147071
:1001B000941901A632FB7F0A28306C2C43AA8B6469
:1001C000A4D30FE522265B4ED78CAB986D397DD337
:1001D000661ADCA54D8599A971963657A56A627194
:1001E0004E5B64A507A55955729561BCF9A4D995D4
:1001F000A7C9E61195905662AB5B5AA26B4ACE2E08
:1002000059732EC1B9BAB5099B4554EB3654AD1498
:10021000BC73DAD48C51482F6E4B534EAEB99A1D35
:100220008E64A645A3FF070618D2CD019BAB69607B
:1002300015D57444F29A55153BEE294B76B5EAE292
:10024000C7BD64C9AA4B18F39425AB2B61CC539658
:10025000AEA9C6564F5932A69A5D237CCE586B5430
:100260000BCFC96DAFDE242A2695BD49610F8D974E
:100270008F745629EC6E55F3698E2644CCADAA399D
:100280009A1471936AE6AC86CDD5E2A6EB92107112
:10029000C99BAE8BD8CDC34DBED3FD7D84093353EE
:1002A000C0F7480AD890F3FF016D184991BC17EFC9
:1002B0006E15A315A2E5939DB57C6C07B67C1CF268
:1002C0001119ACB20E0245287711D90004F0A388A9
:1002D00001BE65B436C88D08F433BB39B4B5E2AE9F
:1002E0000EF2DBD7BAA723D3EA0EF09B8EC8AE92EC
:1002F00024773833F868E6D6F14CD72521E29237D7
:100300005D17B19B879B7CB7FBFB081366A680EF4C
:100310009114B021E7FF036ACE8CF4D49386A549EB
:10032000E231731B962648C625599A1B67ECD434D4
:1003300069EA163133929CA188EC08EA72BA2AA6BF
:100340002DB4CBC9BA19B5D43527EBA929CC679FF1
:10035000AC65E7E09E32AA11D1CDC34D6B7BA054B2
:10036000F54C6768A1C4C4178FA54637975ED2AE17
:1003700012DD5D7A89BB7272F5D8D902A8B2580134
:10038000DF9B09E0B77401FCE6A9809F5205F06786
:10039000FBFF030AC82A5401CDA1A622091B575707
:1003A00035F22C7C9335F32A2BD951D32DABCCFCD1
:1003B0004BC337AF32C9B7725F39CAE8D39B7B7280
:1003C000A9BEE44832270678C655013FA528E0B704
:1003D000520E30E0B7D4FF07A22B202DAA1AAAB6DE
:1003E00081D48872AC808FC43490AA8F44D5434D99
:1003F000CB16338CB644239ADC21A76BAD602883DF
:100400009C9E7582691274B2D1F18774AA894627BD
:100410001836395C179D60A892345BB4A2A6CAD284
:100420007DD18873B6F2A89623CD834D235DB72C7A
:100430000F74F3C8DC8A5CA9A43B55AB73E5E23AC0
:10044000D76D2C498B3D6F95B1784DD77894A664C4
:10045000C333E2529A928D08F34B614A31DCB826DD
:10046000BB250577957AF40606CCA126BB839318A5
:10047000CF4AAD2E31ED3CA72426C354F192648BB4
:100480008A98CB2B2E34532D0E2F57B30C0D3CBC1A
:100490003C4C4BCAF4F0720F6E4953CDCB532D3503
:1004A0004D0F2F0FD70C0D3DBCDC4DD3DDC2F072CC
:1004B000524F579BC3AB89BD422D0FAF5AD171919B
:1004C00055BC2CC53BD865F28294184E3BC1734293
:1004D000323315454F79526A55A6A3FF07C36C8680
:1004E000B3276D0FA748994E553CBC2265364DD1B8
:1004F000F032D3BE34DAC3EB82E2DA6535AF31F2E3
:100500006B9795BC86D86F82A6730BC69E7299CCEA
:10051000CB02AD3C9A1060AB62052C378400A97306
:100520000000FE1F02B83A8C01DFA473400147B9F6
:100530002F333B735F537CEC9AC563D5D175AE5BAB
:10054000FC645C358791F18336B56855C56FDA4533
:100550002D1C2DB738379F603CBC9A85A32566F7C4
:100560008A571CA96756CA5EF0B216B2F189CE8BC3
:100570009225C72B33CF48B199B4F3FF0ED8AEDD27
:10058000030E38A6D201D3B42CAD6A359DB17DDC03
:10059000EEC465D7F1724724B319D9D90570404923
:1005A000EA0298BE4201DFA4694000DF95FC3F02E9
:1005B000E83E8C01DD650860984C063493CE80E6F9
:1005C000DA9A146BAA47D15E56AA6D56CD78D9A98E
:1005D0001C670583E1A4BA38EE16869BFA60875B38
:1005E000186EEE8B1D6E61B9693665BA8DE5E53E14
:1005F0001CE90E969B5BAB952B586ECEE53A6AF3E1
:10060000B835847B05A3E336EF9219B486DBB46971
:10061000B4D12A4E659A99CE28D985714C186D6748
:1006200047C65E534A9CB5E2854526FE7F0C18B648
:100630009A01C3750960D80E0930A09BB6A0BBB063
:10064000AA164E82EBEAA9FA59499E59239A273BEA
:100650007866AE4A9C9CE099D32ABD7292EFE688F8
:10066000E4454D7E982D626737F9A137A76C94E475
:10067000C71EDC3CA5831F8BEB520E0E7E2E4EC791
:1006800031D279A53A0DD9C4FF0702D82E9C01DBDF
:10069000A63360FB3001EC20128CE4D8CA3296738A
:1006A0006341398998C14D0DEDB02A05370FB4A5C6
:1006B000AE5CDC36D0832F4A717B03F73859CDED21
:1006C0001EB46B1435B76B949991D5DC2648774BE3
:1006D00066711B21DB2D8AC96D88FC26283AB7215B
:1006E000F41FA365BC0238BB3D8EF02BE208B73483
:1006F000FF0F0E386E2500A30D3AA037C5A0059E4A
:10070000563586AA5E8CA482B2D774312269AD1C9C
:10071000D3C1D0FA282B2D47C31BC2C4AEC6CD9C73
:1007200048539AFF0FCC677542595D3A4F9D366327
:10073000B759DC305B5C2361F3E21CF1F098C34BEA
:100740007D39CA1D2C2FB715EF7079BCD2467C526B
:10075000E5F14A6AB37147C32D39344B2335B77A73
:1007600055338F59DCA244B5BC66728B64F5F6989C
:10077000C14D42D42762382F4AB69C8868BCA695E2
:10078000F85CA109867791115BFF0FA14A4CF43107
:10079000DD853271B6C774978ACC541FCB5DC933DF
:1007A000357DCCE42D6B20F958EB9FA4CB56136F0D
:1007B00074E2AE375C3DD1899BBD74F1442769E694
:1007C000DAD5139DB4AB9B104F74F22967C23CE598
:1007D00029A7E9AA9054A79ABE3D525A9D66C551D1
:1007E000496B74DA954630A2D1E8662EE4CACA6D28
:1007F0005821893A23872173B5714D6A86202CCE02
:10080000CD891A82B05CB5246A08222A2D3DAB3E00
:100810004AAD34F3F55A4E231EC55833A79EA06A3D
:10082000F1AD9EB2E2EE49AB3ACA2A667294E9DAB9
:10083000BB0AC3308CB51D5B4C42B9BB886C000051
:10084000015C91260104149FFA5A0E08F85C9D0180
:100850005F7808E08B74057C15AE8161576B9ADC7C
:10086000758ED76D48892F3E410BED293AFB44D553
:10087000A787DAA296C45011CAB554AD656A88B884
:100880006A6D0E63C6D6B88DB94638D9EC34E5AC7E
:1008900045BE75C2948478BB37B6939EC82482BB8C
:1008A00088C8060080FF5A7604F8828D030AF8CAC9
:1008B000DC015F7928E0EB30057CEDBEBCAD8A340D
:1008C00062D50D4EB4DC1287771AD528091EBE24D6
:1008D00036A815CADD4564038001F25431C05715AE
:1008E00002F8CA8C01DF5812E01B0B047C2F8680B3
:1008F000EFD4FE5A3608E8D2150302A83A5D015536
:10090000960E3FA570E798BD82DCDB5DADD60A4A46
:10091000F870F586272EFED3C56B9DB4E9AB9468BD
:1009200078AAEA2FC3A3F1E96AD888F0D9A76F6142
:10093000A2DC66AFBE85B6349BB5FAEE5DD273CE4F
:10094000EABB338AAC3A63E85629ABAB94BE674541
:10095000CB9E5DFAE604B37276EA8A266FCF29A9A8
:100960004DCA343D6AC7C10FFF5A5608A8CA940041
:100970005D843120A90A05541D16BCAADCC3C4CE6F
:100980000A92DA94A04DC74F7CDA0B739F20AA2DF0
:1009900073CE759228B723D9F7CA82B916D35CA350
:1009A000887A2A83728D2EEAED08CCD38668B6CD7C
:1009B000297719A3DED6A0DE650C665B82739731BA
:1009C000D82D0BEA53C610B624B8779942984CE557
:1009D000DC6E0AA34CC317FE5A1608A8C28C020488
:1009E000682ADCF9515B96798D10E5CA2E9A7672E9
:1009F000D0C25C252123CD0C4FD4227A46343EF15F
:100A00004886D2B1EA24331662E7AA55ACD404D59D
:100A10008D47B35333E42C69ED4E813053A7F5BBBA
:100A20001443F49236EC9204D54BD2B8AB23F43491
:100A3000CE6319577384AE26699C8DC0AB6B87B1AA
:100A40007B94998AF25A660E5856CB00D7AB19E0C0
:100A500038CBE60C658A61AD869DA579A42D1E6E06
:100A600061699AF6790485A46BC8EF161794A1C141
:100A7000BB5B5E6186057E0AA50A25A6753A348EA3
:100A80005FA8EB4BD749BBE6128FDDE0C578B2BC5F
:100A9000368315EB2EF2480D469E89E92B31C8327C
:100AA0002C9EABFF5A26A69076CC436BB942D83524
:100AB00077A91972E546D26256CBAC9F68E14E2306
:100AC000097123553A9EB8C44B776D74E393547BF8
:100AD000E56E2D4FD6EC5684B53A450D5DA1D6A8EE
:100AE000F4C5588478EC34646D16EA8DC29095662E
:100AF000B1250E43921A439E260C4949B478EA3434
:100B0000161BA6EAB1C92482BB88C80600F82600D5
:100B100000000800020100000304070000000000BC
:100B200000000001020408102040800102040810A7
:100B30002001020408102004040404040404040234
:100B40000202020202030303030303000000002366
:100B5000002600290000000000250028002B0000CE
:100B6000000000240027002A000011241FBECFEF40
:100B7000D8E0DEBFCDBF12E0A0E0B1E0EEE4F3E4E8
:100B800002C005900D92A234B107D9F722E0A2E489
:100B9000B2E001C01D92A73DB207E1F70E94951D8A
:100BA0000C94A5210C9400002F923F924F925F92DB
:100BB0006F927F928F929F92AF92BF92CF92DF926D
:100BC000EF92FF920F931F93CF93DF93CDB7DEB7D2
:100BD0006E970FB6F894DEBF0FBECDBF809157025F
:100BE0008093B40090916A02992309F18091560292
:100BF000891720F48F5F8093560202C0109256022C
:100C0000E0915602E93288F5F0E0E85FFE4FA081FE
:100C10002091680230916902BB27A7FDB0950E9420
:100C20005A21BB27A92F982F872F9C0120C02091E4
:100C3000060130910701A9015695479520FF03C091
:100C400080E098EB02C080E090E0842795279093A5
:100C5000070180930601209168023091690280FDAE
:100C600006C031952195310902C020E030E0C090E6
:100C70005D02DD24C7FCD094E0905202F090530254
:100C800060915C0240915402509155026403C0018E
:100C9000659F900D1124880F892F881F990B281BA1
:100CA000390BCE9CC001CF9C900DDE9C900D112481
:100CB000880F892F881F990B281B390B00915E0222
:100CC000112707FD10958090500290905102089DC9
:100CD000C001099D900D189D900D1124880F892F3A
:100CE000881F990BA901481B590B5C8F4B8F609093
:100CF0005F02772467FC709420904E0230904F0280
:100D0000629CC001639C900D729C900D1124880F11
:100D1000892F881F990B2A01481A590A809160026D
:100D2000682F772767FD70957A83698380914C02DD
:100D300090914D029C838B83FC016E9FC0016F9F3D
:100D4000900D7E9F900D1124880F892F881F990B7D
:100D5000A201481B590B5E834D8380916102682F6D
:100D6000772767FD709578876F8380914A0290910D
:100D70004B029A878987FC016E9FC0016F9F900D7F
:100D80007E9F900D1124880F892F881F990B481B77
:100D9000590B5C874B8780916202482F552747FD8E
:100DA00050955E874D876091480270914902788B1B
:100DB0006F87469FC001479F900D569F900D11244D
:100DC000880F892F881F990BEB85FC85E81BF90B91
:100DD000FA8BE98B80916302482F552747FD509588
:100DE0005C8B4B8B60914602709147027E8B6D8BC2
:100DF000469FC001479F900D569F900D1124880F6C
:100E0000892F881F990B5F01A81AB90A8091640283
:100E100090916502988F8F8BE0914402F09145028A
:100E2000FA8FE98FAC014E9FC0014F9F900D5E9FDE
:100E3000900D1124880F892F881F990BD501A81BAD
:100E4000B90B60916602709167027E8F6D8F409141
:100E5000420250914302649FC001659F900D749FB0
:100E6000900D1124880F892F881F990BBD01681BD5
:100E7000790B611582E078073CF461159EEF7907E4
:100E80002CF460E07EEF02C06FEF71E0C29EC00103
:100E9000C39E900DD29E900D1124880F892F881F1C
:100EA000990B8E0D9F1D9093550280935402EB8DEC
:100EB000FC8D0E9FC0010F9F900D1E9F900D112461
:100EC000880F892F881F990B880D991D90935302C5
:100ED00080935202649CC001659C900D749C900D9F
:100EE0001124880F892F881F990B820D931D9093D1
:100EF00051028093500229813A81ED81FE812E9F1B
:100F0000C0012F9F900D3E9F900D1124880F892FB7
:100F1000881F990B2B813C81820F931F90934F0266
:100F200080934E02EF81F8852B853C85E29FC001BE
:100F3000E39F900DF29F900D1124880F892F881F39
:100F4000990BE985FA858E0F9F1F90934D02809330
:100F50004C022D853E85E989FA892E9FC0012F9F7D
:100F6000900D3E9F900D1124880F892F881F990B9B
:100F70002F853889820F931F90934B0280934A02EA
:100F8000EB89FC89EA9DC001EB9D900DFA9D900DC7
:100F90001124880F892F881F990B2D893E89820F74
:100FA000931F9093490280934802EF89F88DEA9F3E
:100FB000C001EB9F900DFA9F900D1124880F892F8F
:100FC000881F990B298D3A8D820F931F90934702AA
:100FD00080934602ED8DFE8DE69FC001E79F900D48
:100FE000F69F900D1124880F892F881F990B840F6D
:100FF000951F90934502809344027093430260933F
:10100000420275956795759567956058609357028C
:101010006E960FB6F894DEBF0FBECDBFDF91CF91B5
:101020001F910F91FF90EF90DF90CF90BF90AF9006
:101030009F908F907F906F905F904F903F902F90F8
:101040000895E0919002F0E0ED5CFD4F808190E02A
:1010500088319105A0F5FC01EC5CFF4F0C94542104
:101060008FE301C086E085B931C08BE5FCCF8FE40A
:10107000FACF86E6F8CF8DE7F6CF87E0F4CF8FE79B
:10108000F2CF87E6F0CF15B821C089E7ECCF81E336
:10109000EACF8DE6E8CF83E7E6CF88E3E4CF87E7C2
:1010A000E2CF8CE7E0CF89E3DECF88E7DCCF8CE5C9
:1010B000DACF8DE3D8CF80E1D6CF87E3D4CF15B890
:1010C00081E080938C0284E080938D0280918A027B
:1010D000882311F02F9A08952F9808951092AA024C
:1010E0001092A90280918F0290E060E06430B0F429
:1010F000262F30E071E0760FAC01062E02C0559528
:1011000047950A94E2F740FF07C06093A802309326
:10111000AA022093A90204C0672FE8CF6093A80217
:101120002091A9023091AA0280919002880F880F25
:10113000820F8093A302E82FF0E0E559FD4F9081E4
:10114000911146C021E020933102208390E080314C
:101150009105A0F5FC01E45BFF4F0C94542183E062
:1011600001C084E080938E0281E08093890208951B
:1011700082E0F8CF81E080938E02F7CF89E018C03B
:1011800086E016C083E014C085E0ECCF88E010C094
:1011900085E00EC082E00CC08BE080938E0281E07F
:1011A00080938802089587E003C084E001C081E055
:1011B00080938E02089510928E020895109231024B
:1011C00010928E0220938C0284E080938D02089509
:1011D00010923102089515B868EC70E080E090E05C
:1011E0000C94551C15B880E09AE0E82FF0E0ED5C17
:1011F000FD4F90838F5F8930C0F38093A8020895DC
:1012000080E0E82FF0E0E559FD4F10828F5F8131DB
:10121000C0F38093A80208950E94000915B880E0E9
:101220009AE0E82FF0E0ED5CFD4F90838F5F89300E
:10123000C0F38093A80210927F021092C502109210
:10124000C6021092C7021092C80210928102109238
:10125000C1021092C2021092C3021092C4021092F4
:10126000B0021092AF021092AA021092A90210923C
:10127000BD021092BE021092BF021092C0021092E4
:10128000900210928F0210928E021092A50210927C
:10129000A40210928A0210928C0210928D02109277
:1012A00089021092AE021092AD0210928802109242
:1012B000870281E0809331028093850280938402CB
:1012C0001092820210928002109283021092A30266
:1012D00010928B021092330288E08093320214BE87
:1012E00008950C940C09F89481E080938C0282E0BC
:1012F00080938D0214BEE0E6F0E080818F778083DA
:1013000084E090E09093B0028093AF0278941895B7
:10131000F894A895E0E6F0E088E180838FE480838C
:1013200014BE8081877F808378940895CF9362E094
:1013300082E00E94FC1C61E083E00E94FC1C209A79
:10134000219A229A239A249A259A269A279A60E02B
:1013500084E00E94FC1C60E085E00E94FC1C60E0D0
:1013600086E00E94FC1C60E087E00E94FC1C60E0BC
:1013700084E00E94351D60E085E00E94351D60E03C
:1013800086E00E94351D60E087E00E94351D61E027
:101390008EE00E94FC1C61E08FE00E94FC1C61E07A
:1013A00080E10E94FC1C61E081E10E94FC1C61E084
:1013B00082E10E94FC1C61E083E10E94FC1C61E070
:1013C00080E00E94FC1C61E081E00E94FC1C0E9405
:1013D0000009C1E0C09385020E94261C6093B502FB
:1013E0007093B6028093B7029093B80284B78F705F
:1013F00090E09093AA028093A9028091A902909113
:10140000AA02181619061CF5C0938C028091A90235
:101410009091AA028230910559F01CF4019791F045
:101420000BC08430910531F0089731F487E00DC08E
:1014300085E00BC083E009C08091A9029091AA02C7
:1014400080FF02C086E001C089E080938D02809118
:10145000600087FF0BC081E080938C0287E080935F
:101460008D028091600080688093600014BECF91EF
:101470000C948809A89588E10FB6F89480936000D1
:10148000109260000FBE88B18F6388B915B8E4E68A
:10149000F0E08081806880838081826080838081A9
:1014A00084608083EAE7F0E080818F77808380E842
:1014B00080BF43E050E061E779E080E00E945C1B80
:1014C00083B7817F846083BFF89483B7816083BFD3
:1014D0007894889583B78E7F83BF7894E4E6F0E0B4
:1014E00080818F7D808380E00E947C1B88B1807C1E
:1014F00088B90E94261C6093B5027093B60280934F
:10150000B7029093B8020E9488090C940C094F927C
:101510005F926F927F928F929F92AF92BF92CF9283
:10152000DF92EF92FF92CF93DF93FA0115B8ACEB05
:10153000B2E09B01AC010E9461214B015C01BF0143
:10154000882777FD8095982F0E94A91E9B01AC01EA
:1015500060E070E080E89FE30E940E1E20E034E22D
:1015600044E759E40E945D1F0E94761E2B01EB01A7
:1015700077FD2196D595C795C12CD12C760166248F
:1015800057FC6094762CC814D904EA04FB049CF43C
:1015900061E083E00E94351DCE010E948F1C60E057
:1015A00083E00E94351DCE010E948F1CC40CD51C07
:1015B000E61CF71CE8CFDF91CF91FF90EF90DF9012
:1015C000CF90BF90AF909F908F907F906F905F90E3
:1015D0004F9008950F931F9318B815B8E09190029B
:1015E000F0E0E75DFD4F61E080810E94351D409194
:1015F0009002443030F489B182958F7080938F02CD
:1016000002C010928F0280918F02882331F00E94D5
:101610006E0881E0809387021CC0109287024430DC
:10162000C0F4842F90E00196880F991F880F991FAE
:10163000440F440F242F30E051E0540F281739078E
:1016400034F4F901E559FD4F1082452FF3CF409353
:10165000A802809190028F5F883018F480939002E6
:1016600002C0109290028FEF88B9E0919002F0E0F2
:10167000E75DFD4F60E080810E94351D8CE291E0C6
:101680000E948F1C8091A402E09190028E1304C0EE
:1016900081E080938A0202C010928A02F0E0ED5C41
:1016A000FD4F80818A3028F080918C02882309F4D4
:1016B000AFC00E94210880E991E00E948F1C82E067
:1016C0000E946B1D21E0892B09F420E02093860203
:1016D00021119BC081E08093830280938402109249
:1016E000C1021092C2021092C3021092C402109260
:1016F000820210928B020E94261C6093B1027093AA
:10170000B2028093B3029093B40215B864E670E01D
:1017100080E090E00E94551C82E00E946B1D21E059
:10172000892B09F420E020938602222379F30E947A
:10173000261C0091B1021091B2022091B3023091A7
:10174000B402601B710B820B930B693E73408105E1
:10175000910558F148E853E16AE070E080E090E0DC
:101760000E94870A80913D02882319F010923D0261
:101770001CC011E010933D0248E853E160E570E0C1
:1017800080E090E00E94870A80913C02882319F053
:1017900010923C020AC040E45FE160E570E080E046
:1017A00090E00E94870A10933C020E94261C6093DE
:1017B000B5027093B6028093B7029093B8028091FD
:1017C000AF029091B00201979093B0028093AF0264
:1017D0008091AF029091B00297FD28C08091AF0236
:1017E0009091B002029711F180918C0281111EC07C
:1017F0001092C1021092C2021092C3021092C4024F
:101800001092A5021092900222C0109283021FC073
:1018100015B880919002873009F04DCF80918B02EE
:10182000882309F448CF80E485B945CF0E940C098C
:101830001092330281E09AE0E82FF0E0ED5CFD4F7A
:1018400090838F5F8830C0F38093A802D1CF1F911F
:101850000F910895CF92DF92EF92FF926B017C017E
:101860001092BD021092BE021092BF021092C002EE
:1018700010927E026093B9027093BA028093BB0209
:101880009093BC0220E836E948E950E00E943521F7
:101890002093BD023093BE024093BF025093C0021A
:1018A0008091BD029091BE02A091BF02B091C00292
:1018B000181619061A061B064CF48091BD02909169
:1018C000BE02A091BF02B091C0020FC08091BD02C4
:1018D0009091BE02A091BF02B091C002B095A095B8
:1018E000909581959F4FAF4FBF4F8093BD029093CE
:1018F000BE02A093BF02B093C0028091BD0290913E
:10190000BE02A091BF02B091C002181619061A06B5
:101910001B0654F581E080937E0287E08093A70246
:101920008091BD029091BE02A091BF02B091C00211
:101930008093A2022091BD023091BE024091BF026D
:101940005091C00260E879E687E69FEF0E9425216A
:101950006C0D7D1D8E1D9F1D6093B9027093BA02A0
:101960008093BB029093BC02C090B902D090BA029F
:10197000E090BB02F090BC02C701B60120E432E463
:101980004FE050E00E9435212093BD023093BE020B
:101990004093BF025093C0028091BD029091BE025D
:1019A000A091BF02B091C002181619061A061B06B4
:1019B0004CF48091BD029091BE02A091BF02B09103
:1019C000C0020FC08091BD029091BE02A091BF02E3
:1019D000B091C002B095A095909581959F4FAF4F63
:1019E000BF4F8093BD029093BE02A093BF02B093FD
:1019F000C0028091BD029091BE02A091BF02B09141
:101A0000C00220917E02181619061A061B0614F051
:101A1000222361F1211103C086E08093A70281E0B7
:101A200080937E028091BD029091BE02A091BF0280
:101A3000B091C0028093A1022091BD023091BE02FC
:101A40004091BF025091C00260EC7DEB80EF9FEFB0
:101A50000E9425216C0D7D1D8E1D9F1D6093B90276
:101A60007093BA028093BB029093BC02C090B902FB
:101A7000D090BA02E090BB02F090BC02C701B60160
:101A800020EA36E841E050E00E9435212093BD0273
:101A90003093BE024093BF025093C0028091BD02BA
:101AA0009091BE02A091BF02B091C0021816190613
:101AB0001A061B064CF48091BD029091BE02A091C3
:101AC000BF02B091C0020FC08091BD029091BE02D2
:101AD000A091BF02B091C002B095A095909581955C
:101AE0009F4FAF4FBF4F8093BD029093BE02A09314
:101AF000BF02B093C0028091BD029091BE02A0913E
:101B0000BF02B091C00220917E02181619061A0673
:101B10001B0614F0222361F1211103C085E080939C
:101B2000A70281E080937E028091BD029091BE0267
:101B3000A091BF02B091C0028093A0022091BD028B
:101B40003091BE024091BF025091C00260E679E739
:101B50008EEF9FEF0E9425216C0D7D1D8E1D9F1D18
:101B60006093B9027093BA028093BB029093BC0257
:101B7000C090B902D090BA02E090BB02F090BC02D3
:101B8000C701B60120E137E240E050E00E94352174
:101B90002093BD023093BE024093BF025093C00217
:101BA0008091BD029091BE02A091BF02B091C0028F
:101BB000181619061A061B064CF48091BD02909166
:101BC000BE02A091BF02B091C0020FC08091BD02C1
:101BD0009091BE02A091BF02B091C002B095A095B5
:101BE000909581959F4FAF4FBF4F8093BD029093CB
:101BF000BE02A093BF02B093C0028091BD0290913B
:101C0000BE02A091BF02B091C00220917E021816C0
:101C100019061A061B0614F0222351F1211103C0E4
:101C200084E08093A70281E080937E028091BD02D0
:101C30009091BE02A091BF02B091C00280939F021A
:101C40002091BD023091BE024091BF025091C0026E
:101C5000A0EFB8ED0E946F216C0D7D1D8E1D9F1DA4
:101C60006093B9027093BA028093BB029093BC0256
:101C7000C090B902D090BA02E090BB02F090BC02D2
:101C8000C701B60128EE33E040E050E00E94352164
:101C90002093BD023093BE024093BF025093C00216
:101CA0008091BD029091BE02A091BF02B091C0028E
:101CB000181619061A061B064CF48091BD02909165
:101CC000BE02A091BF02B091C0020FC08091BD02C0
:101CD0009091BE02A091BF02B091C002B095A095B4
:101CE000909581959F4FAF4FBF4F8093BD029093CA
:101CF000BE02A093BF02B093C0028091BD0290913A
:101D0000BE02A091BF02B091C00220917E021816BF
:101D100019061A061B0614F0222351F1211103C0E3
:101D200083E08093A70281E080937E028091BD02D0
:101D30009091BE02A091BF02B091C00280939E021A
:101D40002091BD023091BE024091BF025091C0026D
:101D5000A8E1BCEF0E946F216C0D7D1D8E1D9F1DA3
:101D60006093B9027093BA028093BB029093BC0255
:101D7000C090B902D090BA02E090BB02F090BC02D1
:101D8000C701B60124E630E040E050E00E94352172
:101D90002093BD023093BE024093BF025093C00215
:101DA0008091BD029091BE02A091BF02B091C0028D
:101DB000181619061A061B064CF48091BD02909164
:101DC000BE02A091BF02B091C0020FC08091BD02BF
:101DD0009091BE02A091BF02B091C002B095A095B3
:101DE000909581959F4FAF4FBF4F8093BD029093C9
:101DF000BE02A093BF02B093C0028091BD02909139
:101E0000BE02A091BF02B091C00220917E021816BE
:101E100019061A061B0614F0222351F1211103C0E2
:101E200082E08093A70281E080937E028091BD02D0
:101E30009091BE02A091BF02B091C00280939D021A
:101E40002091BD023091BE024091BF025091C0026C
:101E5000ACE9BFEF0E946F216C0D7D1D8E1D9F1D93
:101E60006093B9027093BA028093BB029093BC0254
:101E7000C090B902D090BA02E090BB02F090BC02D0
:101E8000C701B6012AE030E040E050E00E94352171
:101E90002093BD023093BE024093BF025093C00214
:101EA0008091BD029091BE02A091BF02B091C0028C
:101EB000181619061A061B064CF48091BD02909163
:101EC000BE02A091BF02B091C0020FC08091BD02BE
:101ED0009091BE02A091BF02B091C002B095A095B2
:101EE000909581959F4FAF4FBF4F8093BD029093C8
:101EF000BE02A093BF02B093C0028091BD02909138
:101F0000BE02A091BF02B091C00220917E021816BD
:101F100019061A061B0614F0222351F1211103C0E1
:101F200081E08093A70281E080937E028091BD02D0
:101F30009091BE02A091BF02B091C00280939C021A
:101F40002091BD023091BE024091BF025091C0026B
:101F5000A6EFBFEF0E946F216C0D7D1D8E1D9F1D92
:101F60006093B9027093BA028093BB029093BC0253
:101F700080917E02811102C01092A7028091B90265
:101F800080939B021092BD021092BE021092BF027B
:101F90001092C002FF90EF90DF90CF900895CF9203
:101FA000DF92EF92FF926B017C011092BD021092C2
:101FB000BE021092BF021092C0021092A60281E0EF
:101FC000E82FF0E0EF56FD4F10828F5F8730C0F3AF
:101FD0008093A802C092B902D092BA02E092BB02EA
:101FE000F092BC02C701B60120EA36E841E050E0B9
:101FF0000E9435212093BD023093BE024093BF0260
:102000005093C0028091BD029091BE02A091BF0288
:10201000B091C002181619061A061B064CF48091DE
:10202000BD029091BE02A091BF02B091C0020FC04C
:102030008091BD029091BE02A091BF02B091C002FA
:10204000B095A095909581959F4FAF4FBF4F8093CE
:10205000BD029093BE02A093BF02B093C0028091D4
:10206000BD029091BE02A091BF02B091C0021816AD
:1020700019061A061B063CF581E08093A6028091A2
:10208000BD029091BE02A091BF02B091C0028093A8
:1020900092022091BD023091BE024091BF02509148
:1020A000C00260E679E78EEF9FEF0E9425216C0D5C
:1020B0007D1D8E1D9F1D6093B9027093BA0280939F
:1020C000BB029093BC02C090B902D090BA02E090DB
:1020D000BB02F090BC02C701B60120E137E240E04C
:1020E00050E00E9435212093BD023093BE02409300
:1020F000BF025093C0028091BD029091BE02A09198
:10210000BF02B091C002181619061A061B064CF43D
:102110008091BD029091BE02A091BF02B091C00219
:102120000FC08091BD029091BE02A091BF02B091FC
:10213000C002B095A095909581959F4FAF4FBF4F2E
:102140008093BD029093BE02A093BF02B093C002E1
:102150008091BD029091BE02A091BF02B091C002D9
:10216000181619061A061B062CF582E08093A602A3
:102170008091BD029091BE02A091BF02B091C002B9
:10218000809393022091BD023091BE024091BF0224
:102190005091C002A0EFB8ED0E946F216C0D7D1D23
:1021A0008E1D9F1D6093B9027093BA028093BB028B
:1021B0009093BC02C090B902D090BA02E090BB02EA
:1021C000F090BC02C701B60128EE33E040E050E0D9
:1021D0000E9435212093BD023093BE024093BF027E
:1021E0005093C0028091BD029091BE02A091BF02A7
:1021F000B091C002181619061A061B064CF48091FD
:10220000BD029091BE02A091BF02B091C0020FC06A
:102210008091BD029091BE02A091BF02B091C00218
:10222000B095A095909581959F4FAF4FBF4F8093EC
:10223000BD029093BE02A093BF02B093C0028091F2
:10224000BD029091BE02A091BF02B091C0021816CB
:1022500019061A061B062CF583E08093A6028091CE
:10226000BD029091BE02A091BF02B091C0028093C6
:1022700094022091BD023091BE024091BF02509164
:10228000C002A8E1BCEF0E946F216C0D7D1D8E1D68
:102290009F1D6093B9027093BA028093BB02909322
:1022A000BC02C090B902D090BA02E090BB02F0909C
:1022B000BC02C701B60124E630E040E050E00E94D5
:1022C00035212093BD023093BE024093BF0250934C
:1022D000C0028091BD029091BE02A091BF02B09158
:1022E000C002181619061A061B064CF48091BD028E
:1022F0009091BE02A091BF02B091C0020FC0809128
:10230000BD029091BE02A091BF02B091C002B095F3
:10231000A095909581959F4FAF4FBF4F8093BD0281
:102320009093BE02A093BF02B093C0028091BD0201
:102330009091BE02A091BF02B091C002181619067A
:102340001A061B062CF584E08093A6028091BD023C
:102350009091BE02A091BF02B091C00280939502FD
:102360002091BD023091BE024091BF025091C00247
:10237000ACE9BFEF0E946F216C0D7D1D8E1D9F1D6E
:102380006093B9027093BA028093BB029093BC022F
:10239000C090B902D090BA02E090BB02F090BC02AB
:1023A000C701B6012AE030E040E050E00E9435214C
:1023B0002093BD023093BE024093BF025093C002EF
:1023C0008091BD029091BE02A091BF02B091C00267
:1023D000181619061A061B064CF48091BD0290913E
:1023E000BE02A091BF02B091C0020FC08091BD0299
:1023F0009091BE02A091BF02B091C002B095A0958D
:10240000909581959F4FAF4FBF4F8093BD029093A2
:10241000BE02A093BF02B093C0028091BD02909112
:10242000BE02A091BF02B091C002181619061A068A
:102430001B062CF585E08093A6028091BD02909149
:10244000BE02A091BF02B091C0028093960220917B
:10245000BD023091BE024091BF025091C002A6EF72
:10246000BFEF0E946F216C0D7D1D8E1D9F1D60931F
:10247000B9027093BA028093BB029093BC02809120
:10248000B9029091BA02A091BB02B091BC02181699
:1024900019061A061B062CF426E02093A602809348
:1024A00097021092BD021092BE021092BF021092CB
:1024B000C002FF90EF90DF90CF9008958F929F928F
:1024C000AF92BF92CF92DF92EF92FF920F931F9342
:1024D000CF93DF9300D000D0CDB7DEB76091C502B7
:1024E0007091C6028091C7029091C80220E030E04E
:1024F000A9010E940A1E87FF04C081E080938B021D
:1025000002C010928B026091C5027091C602809148
:10251000C7029091C80220E030E0A9010E94591F33
:1025200018164CF48091C5029091C602A091C70282
:10253000B091C80209C08091C5029091C602A091D5
:10254000C702B091C802B0588093C5029093C602EA
:10255000A093C702B093C8021092BD021092BE02AF
:102560001092BF021092C0026091C5027091C60223
:102570008091C7029091C8020E94761E6093BD02AE
:102580007093BE028093BF029093C0026091BD021F
:102590007091BE028091BF029091C0020E942A0CED
:1025A000C090C502D090C602E090C702F090C80269
:1025B0006091C5027091C6028091C7029091C802D5
:1025C0000E94761E0E94A91E9B01AC01C701B601A4
:1025D0000E94A51D6093C5027093C6028093C70236
:1025E0009093C8026091C5027091C6028091C702A3
:1025F0009091C80220E034E244E759E40E945D1F54
:102600006093C5027093C6028093C7029093C8027C
:10261000C090C502D090C602E090C702F090C802F8
:102620006091C5027091C6028091C7029091C80264
:102630000E94761E0E94A91E9B01AC01C701B60133
:102640000E94A51D20E030E040E05FE30E94591F9A
:1026500018167CF46091C5027091C6028091C70281
:102660009091C8020E94761E6F5F7F4F8F4F9F4FE1
:102670000AC06091C5027091C6028091C702909114
:10268000C8020E94761E6093BD027093BE028093C2
:10269000BF029093C0028091BD029091BE02A091B2
:1026A000BF02B091C002181619061A061B065CF488
:1026B0006091BD027091BE028091BF029091C002F4
:1026C0000E94CF0F02C01092A60280E09AE0E82F8D
:1026D000F0E0ED5CFD4F90838F5F8830C0F3109287
:1026E000BD021092BE021092BF021092C002109260
:1026F000C5021092C6021092C7021092C80281E071
:1027000090E0A0E0B0E08093B9029093BA02A09369
:10271000BB02B093BC021092A8029090A702AA2418
:10272000A394B12C00E010E0812CE82DF0E0DF0153
:10273000A656BD4F1196AC91ED5CFD4FA083C090A5
:10274000BD02D090BE02E090BF02F090C002B0E0A7
:102750009501A8010E946121C60ED71EE81EF91E30
:10276000C092BD02D092BE02E092BF02F092C002BF
:10277000AAE0B0E00E94612121E0280D921620F02D
:10278000822E5B018C01D1CF2093A8026093B90205
:102790007093BA028093BB029093BC021092A40281
:1027A000B090A602B1103DC06091BD027091BE0212
:1027B0008091BF029091C0022091C5023091C60263
:1027C0004091C7025091C80229833A834B835C83AE
:1027D0000E94A91E29813A814B815C810E94A61D1D
:1027E0006093C5027093C6028093C7029093C8029B
:1027F0001092BD021092BE021092BF021092C0024F
:102800000F900F900F900F90DF91CF911F910F912C
:10281000FF90EF90DF90CF90BF90AF909F908F9000
:10282000089588E090E09093AA028093A902809195
:102830008B02882349F08091A9029091AA02019706
:102840009093AA028093A9028091A9029091AA0272
:10285000292D30E020953095820F931F9093AA0286
:102860008093A9028091A9029091AA0218161906D4
:102870000CF09ACF8091A9029091AA022B2D30E002
:10288000281739072CF08091A9029091AA02B82E3E
:10289000B092A60281E08093A80201E0B01618F47D
:1028A0000093A80281CFEAE3F2E0ABE3B2E08291C9
:1028B0008E9382E0E333F807D1F78091A4028F5F13
:1028C0008093A402E02FF0E0EF56FD4F10811093AB
:1028D0003302602F70E080E090E00E94A71E9B0111
:1028E000AC0160E070E080E291E40E94C01F9B01B7
:1028F000AC01C090C502D090C602E090C702F09033
:10290000C802612F70E080E090E029833A834B8316
:102910005C830E94A71E29813A814B815C810E94C1
:102920000E1EA70196010E94A61D6093C50270931A
:10293000C6028093C7029093C8020F5FAFCF829503
:10294000282F237394E0299F90011124982F9C7CB9
:1029500096959695922B892F8575880F9A7A9695DC
:10296000892B0895CF92DF92EF92FF920F931F93DE
:10297000CF93DF93C82EC0915902D0915A02FE0125
:1029800084910E949F14082F10E0102F0027D090F0
:102990005802EC2CF12C97012D0D311D29303105F9
:1029A00034F0FE01319684910E949F14082B0D2C67
:1029B00002C0000F111F0A94E2F720E130E02E1947
:1029C0003F0902C0169507952A95E2F78C2D8D0DCB
:1029D000883018F48093580208C0885080935802B9
:1029E0002196D0935A02C0935902802FDF91CF9144
:1029F0001F910F91FF90EF90DF90CF900895E1E845
:102A0000F0E080E180831092800021E02093CB02EF
:102A100084EF91E09093CD028093CC029093870055
:102A20008093860081E1808384ED95E09093CA02D3
:102A30008093C90220936F0083E28093B0002093BB
:102A4000B1001092700020935B0208951092B000C4
:102A50001092B1001092700010925B0210926F0001
:102A600060E083E00C94351DCF93DF93EC0115B843
:102A700010926F000E94FF1480915B02811102C0CE
:102A80000E94FF14D0935A02C09359021092580228
:102A900084E00E94B214C82F811105C0109269020F
:102AA00010926802ABC08F30E9F410926902109264
:102AB00068021092670210926602109265021092EC
:102AC00064021092630210926202109261021092EC
:102AD000600210925F0210925E0210925D021092EC
:102AE0005C028CC0E82FF0E0E75EFD4F808190E053
:102AF000909369028093680281E00E94B214D82FFB
:102B000086E00E94B214E82FF0E0E752FE4F808189
:102B100080936A02D11172C085E00E94B214E82F3E
:102B2000F0E0E754FE4F8081992787FD90959093C0
:102B300067028093660285E00E94B214E82FF0E0FD
:102B4000E756FE4F8081992787FD90959093650207
:102B50008093640284E00E94B214E82FF0E0E7570B
:102B6000FE4F80818093630284E00E94B214E82FBC
:102B7000F0E0E758FE4F80818093620280916A0204
:102B80008823E1F184E00E94B214E82FF0E0E759D5
:102B9000FE4F80818093610284E00E94B214E82F8E
:102BA000F0E0E75AFE4F80818093600284E00E944B
:102BB000B214E82FF0E0E75BFE4F808180935F0264
:102BC00083E00E94B214E82FF0E0EF5BFE4F8081BB
:102BD00080935E0283E00E94B214E82FF0E0E75C8D
:102BE000FE4F808180935D0283E00E94B214E82F43
:102BF000F0E0EF5CFE4F808180935C0269E170E061
:102C000080E090E00E94551CCF3009F041CFDF9169
:102C1000CF910C942615CF93DF93EC010E94880985
:102C200080913D02882309F454C080913C0288239E
:102C300021F1CC30D10508F04CC0FE01E45AFF4F21
:102C40000C94542185E297E040C082EF96E03DC0AD
:102C50008AE896E03AC08DE296E037C08FEA95E0C8
:102C600034C08CE795E031C084E295E02EC08DED54
:102C700094E02BC089E694E028C0CC30D10548F51B
:102C8000FE01E859FF4F0C94542188ED93E01DC0DC
:102C900086EA9AE01AC087E49AE017C08AED99E0C4
:102CA00014C08BE699E011C085EF98E00EC088EA69
:102CB00098E00BC08BE498E008C087E198E005C07D
:102CC0008BE897E002C08AE691E0DF91CF910C9407
:102CD0003415DF91CF9108958F929F92AF92BF925A
:102CE000CF92DF92EF92FF920F931F93CF93DF93D8
:102CF00000D000D0CDB7DEB7A8950E94261CC090AA
:102D0000B502D090B602E090B702F090B8026C190C
:102D10007D098E099F0969397A438105910510F073
:102D20000E943A0A0E94EA0A80918C02882331F0BC
:102D300084E090E09093B0028093AF02809187028C
:102D4000882371F180913D02882351F1809189029D
:102D5000811105C080918E0290E00E940B16809137
:102D600089028823E9F080918E02833091F038F453
:102D7000813061F08230A1F487E193E00FC08430AC
:102D800059F0853069F489EA92E008C083E993E05C
:102D900005C087EB91E002C087E292E00E94341503
:102DA0008091AF029091B0028230910509F411C276
:102DB00034F4009761F0019709F4F7C030C4833010
:102DC000910509F436C3049709F4BFC328C4809160
:102DD0008702882309F437C40E94261C6093B50239
:102DE0007093B6028093B7029093B802809131023B
:102DF000882309F428C49091890280918502911159
:102E00007AC0882379F080918E02882359F00E943D
:102E1000F208109285021092A4028091880281111A
:102E2000109233021091A502909132028091880293
:102E3000191708F059C090918502911155C0811160
:102E400053C088E0E82FF0E0ED5CFD4FDF01119703
:102E50009C9190838150B1F71092A802C0908E028D
:102E6000C092330200917F02D12CE12CF12C00237F
:102E700009F42DC16091A40270E080E090E00E940E
:102E8000A71E20E030E040E85FE30E94A61D9B0102
:102E9000AC0160E070E080E291E40E94C01F9B0101
:102EA000AC018090C5029090C602A090C702B0907D
:102EB000C802C701B60129833A834B835C830E9411
:102EC000A71E29813A814B815C810E940E1EA501BB
:102ED00094010E94A61D6093C5027093C602809360
:102EE000C7029093C8020BC1882309F4ACC381E0E8
:102EF00080937F0216C1882349F080918E02823030
:102F000009F0ECC281E0809380021FC10E94EB08AF
:102F100010918E02153009F4E1C281E090E09093A7
:102F2000B0028093AF026091BD027091BE028091A9
:102F3000BF029091C0022091C5023091C60240911B
:102F4000C7025091C80229833A834B835C830E9455
:102F5000A91E29813A814B815C810E94A61D609344
:102F6000C5027093C6028093C7029093C802109264
:102F7000BD021092BE021092BF021092C0021092C7
:102F8000C1021092C2021092C3021092C40281E0E8
:102F900080938402109282021092A502812F90E009
:102FA0009093AE028093AD0299C2809187028823EC
:102FB00009F449C30E94261C6093B5027093B602BF
:102FC0008093B7029093B80280913102882309F46C
:102FD0003AC390918902809184029111A8C08823FC
:102FE000A9F080918E02882389F00E94F208109245
:102FF000840280918202811102C010928B02109291
:10300000A402809188028111109233021091A502CE
:103010009091320280918802191708F07CC090913B
:103020008402911178C0811176C088E0E82FF0E029
:10303000ED5CFD4FDF0111979C9190838150B1F7BA
:103040001092A802C0908E02C092330200918102B9
:10305000D12CE12CF12C0023D1F16091A40270E07D
:1030600080E090E00E94A71E20E030E040E85FE3AF
:103070000E94A61D9B01AC0160E070E080E291E43B
:103080000E94C01F9B01AC018090C1029090C202BF
:10309000A090C302B090C402C701B60129833A834D
:1030A0004B835C830E94A71E29813A814B815C81FE
:1030B0000E940E1EA50194010E94A61D6093C102EC
:1030C0007093C2028093C3029093C40218C02091EF
:1030D000BD023091BE024091BF025091C002AAE0F1
:1030E000B0E00E9461216C0D7D1D8E1D9F1D6093BF
:1030F000BD027093BE028093BF029093C0021F5F17
:103100001093A502002309F49EC28091A4028F5F50
:103110008093A40298C2882309F495C281E0809329
:1031200081021092880286E0809332028CC288234A
:1031300091F080918E02823009F0D0C10E94F20895
:103140001092330281E08093820280938B0286E0AA
:1031500080933202C3C10E94EB0880918E028530B9
:1031600019F410927D0208C091E090937D0290E0E6
:103170009093AC028093AB021092890282E090E0BF
:103180009093B0028093AF026091BD027091BE0235
:103190008091BF029091C0022091C1023091C20281
:1031A0004091C3025091C40229833A834B835C83CC
:1031B0000E94A91E29813A814B815C810E94A61D33
:1031C0006093C1027093C2028093C3029093C402C1
:1031D00055C1809182028823A9F02091C1023091CB
:1031E000C2024091C3025091C40260E070E0CB0182
:1031F0000E94A51D6093C1027093C2028093C30216
:103200009093C402809180028823A9F02091C50286
:103210003091C6024091C7025091C80260E070E050
:10322000CB010E94A51D6093C5027093C6028093D6
:10323000C7029093C8028091AD029091AE02823095
:10324000910581F1B4F4019709F05AC06091C5026B
:103250007091C6028091C7029091C8022091C1026C
:103260003091C2024091C3025091C4020E94A61D37
:103270002BC08330910589F1049709F041C060911A
:10328000C5027091C6028091C7029091C802209138
:10329000C1023091C2024091C3025091C4020E9407
:1032A0005D1F12C06091C5027091C6028091C70275
:1032B0009091C8022091C1023091C2024091C30294
:1032C0005091C4020E94A51D6093C5027093C6026E
:1032D0008093C7029093C80227C06091C502709185
:1032E000C6028091C7029091C8022091C10230911C
:1032F000C2024091C3025091C4020E940E1EE4CF4C
:1033000080E090E0A0E8BFE38093C5029093C602FE
:10331000A093C702B093C8020E940C0981E0809379
:103320008C0284E080938D028091C5029091C60248
:10333000A091C702B091C8026091C5027091C60207
:103340008091C7029091C8020E94761E6130764338
:103350008546944C0CF46CC10E945E1280918B02E5
:10336000882341F080913D02882321F087E193E09A
:103370000E9434150BE312E087E0E82EF12CF801EF
:1033800082918F0190E00E940B168091A40290E040
:103390008E159F0531F480913D02882311F0E110D4
:1033A0004DC1F1E0EF1AF10850F780918B028823AC
:1033B00019F081E08093800280917D02882351F191
:1033C00010927D028091AB029091AC029093AE027C
:1033D0008093AD021092C1021092C2021092C302F9
:1033E0001092C40281E080938402109282021092B3
:1033F00081021092A5021092BD021092BE0210929C
:10340000BF021092C00281E090E09093B0028093DE
:10341000AF0219C183E090E09093B0028093AF02B5
:103420001092BD021092BE021092BF021092C00212
:103430000AC180918702882309F405C10E94261CD5
:103440006093B5027093B6028093B7029093B8026E
:1034500080913102882309F4F6C080918902882383
:1034600009F43FC00E94EB0880918E02853099F4E8
:1034700082E090E09093B0028093AF021092BD0280
:103480001092BE021092BF021092C0021092A502CA
:103490000E94F20823C090E09093AE028093AD02A8
:1034A00081E090E09093B0028093AF021092BD0251
:1034B0001092BE021092BF021092C0021092C1027E
:1034C0001092C2021092C3021092C402809384022E
:1034D00010928202109281021092A502109289022B
:1034E000B2C00E94F208109285021092BD021092A2
:1034F000BE021092BF021092C0021092B00210924F
:10350000AF021092A40280918802882351F0109299
:10351000330281E08093A40280937F02109288029C
:1035200092C020918E02822F90E0A0E0B0E08093C4
:10353000BD029093BE02A093BF02B093C00220933D
:10354000330281E08093A5027EC080918D0283309A
:1035500071F1D0F4813009F04CC08BE080933302DC
:1035600085E18093340287E18093350280E1809386
:1035700036028CE0809337028AE080933802109202
:10358000390210923A025FC0853011F1863089F518
:103590008AE0809333028093340292E19093350263
:1035A0002FE02093360220E12093370231C084E1DE
:1035B000809333028FE0809334028AE08093350257
:1035C00093E19093360290E19093370291E120C00D
:1035D00093E1909333029BE0909334028093350201
:1035E000909336028CE0809337028AE08093380211
:1035F00011C080918D02809333028AE0809334025F
:10360000809335029CE090933602909337029BE0C2
:10361000909338028093390280933A0214C00E943A
:103620000C0981E080938C0284E080938D020BC0B2
:1036300081E080938C0280938D028ECE8AE691E0A9
:103640000E943415AECE0F900F900F900F90DF9127
:10365000CF911F910F91FF90EF90DF90CF90BF908F
:10366000AF909F908F9008951F920F920FB60F9278
:1036700011242F933F934F935F936F937F938F9377
:103680009F93AF93BF93EF93FF93E091C902F091A3
:10369000CA020995FF91EF91BF91AF919F918F91D0
:1036A0007F916F915F914F913F912F910F900FBE3E
:1036B0000F901F90189508958230E8F4E82FF0E0FD
:1036C000EE0FFF1FE25CFD4F71836083813041F09C
:1036D000809169008C7F842B80936900E89A08951B
:1036E00080916900440F551F440F551F837F842B21
:1036F00080936900E99A0895823078F4813011F05E
:10370000E89801C0E998E82FF0E0EE0FFF1FE25CB7
:10371000FD4F8BE59BE19183808308951F920F926B
:103720000FB60F9211242F933F934F935F936F9394
:103730007F938F939F93AF93BF93EF93FF93E0910A
:103740003E02F0913F020995FF91EF91BF91AF9139
:103750009F918F917F916F915F914F913F912F91A9
:103760000F900FBE0F901F9018951F920F920FB6DB
:103770000F9211242F933F934F935F936F937F93F7
:103780008F939F93AF93BF93EF93FF93E09140028A
:10379000F09141020995FF91EF91BF91AF919F91F7
:1037A0008F917F916F915F914F913F912F910F90EA
:1037B0000FBE0F901F9018951F920F920FB60F9289
:1037C00011242F933F938F939F93AF93BF93809137
:1037D000CF029091D002A091D102B091D20230914B
:1037E000CE0226E0230F2D3720F40296A11DB11D35
:1037F00005C029E8230F0396A11DB11D2093CE0219
:103800008093CF029093D002A093D102B093D202C2
:103810008091D3029091D402A091D502B091D602AA
:103820000196A11DB11D8093D3029093D402A09361
:10383000D502B093D602BF91AF919F918F913F91E6
:103840002F910F900FBE0F901F9018952FB7F894DF
:103850006091CF027091D0028091D1029091D202FA
:103860002FBF08953FB7F8948091D3029091D4026E
:10387000A091D502B091D60226B5A89B05C02F3FD6
:1038800019F00196A11DB11D3FBF6627782F892F22
:103890009A2F620F711D811D911D43E0660F771FE6
:1038A000881F991F4A95D1F708958F929F92AF92E2
:1038B000BF92CF92DF92EF92FF926B017C010E9448
:1038C000321C4B015C01C114D104E104F104F1F09C
:1038D0000E94A41D0E94321C681979098A099B095B
:1038E000683E73408105910570F321E0C21AD1084A
:1038F000E108F10888EE880E83E0981EA11CB11C37
:10390000C114D104E104F10429F7DDCFFF90EF9059
:10391000DF90CF90BF90AF909F908F9008958330AD
:10392000910528F0880F991F04970197F1F70895E2
:10393000789484B5826084BD84B5816084BD85B58A
:10394000826085BD85B5816085BDEEE6F0E0808151
:1039500081608083E1E8F0E0108280818260808372
:10396000808181608083E0E8F0E0808181608083F5
:10397000E1EBF0E0808184608083E0EBF0E0808127
:1039800081608083EAE7F0E08081846080838081C9
:103990008260808380818E7F808380818068808345
:1039A0001092C1000895833081F028F4813099F09D
:1039B0008230A1F008958730A9F08830B9F08430C2
:1039C000D1F4809180008F7D03C0809180008F773B
:1039D00080938000089584B58F7702C084B58F7D71
:1039E00084BD08958091B0008F7703C08091B000AE
:1039F0008F7D8093B0000895CF93DF9390E0FC011A
:103A0000ED5DF44F2491FC01E95CF44F849188232F
:103A100049F190E0880F991FFC01E15AF44FA591FC
:103A2000B4918B5A944FFC01C591D4919FB7611109
:103A300008C0F8948C91209582238C9388818223EE
:103A40000AC0623051F4F8948C91322F3095832360
:103A50008C938881822B888304C0F8948C91822B6C
:103A60008C939FBFDF91CF9108950F931F93CF93B6
:103A7000DF931F92CDB7DEB7282F30E0F901E15F69
:103A8000F44F8491F901ED5DF44F1491F901E95C73
:103A9000F44F04910023C9F0882321F069830E9428
:103AA000D31C6981E02FF0E0EE0FFF1FEB5AF44FBB
:103AB000A591B4919FB7F8948C91611103C01095B2
:103AC000812301C0812B8C939FBF0F90DF91CF91F9
:103AD0001F910F910895CF93DF93282F30E0F901C4
:103AE000E15FF44F8491F901ED5DF44FD491F90158
:103AF000E95CF44FC491CC2391F081110E94D31C56
:103B0000EC2FF0E0EE0FFF1FE55BF44FA591B491B1
:103B10002C912D2381E090E021F480E002C080E030
:103B200090E0DF91CF91089508950E94981C0E9423
:103B3000941D0E949609C0E0D0E00E946C16209768
:103B4000E1F30E940000F9CF08955058BB27AA273F
:103B50000ED075C166D130F06BD120F031F49F3FAB
:103B600011F41EF45BC10EF4E095E7FB51C1E92F9F
:103B700077D180F3BA17620773078407950718F0A7
:103B800071F49EF58FC10EF4E0950B2EBA2FA02D87
:103B90000B01B90190010C01CA01A0011124FF27FA
:103BA000591B99F0593F50F4503E68F11A16F040F5
:103BB000A22F232F342F4427585FF3CF46953795F4
:103BC0002795A795F0405395C9F77EF41F16BA0BB9
:103BD000620B730B840BBAF09150A1F0FF0FBB1F67
:103BE000661F771F881FC2F70EC0BA0F621F731FB0
:103BF000841F48F4879577956795B795F7959E3F0D
:103C000008F0B3CF9395880F08F09927EE0F97959A
:103C100087950895D9D008F481E008950CD00FC19C
:103C200007D140F0FED030F021F45F3F19F0F0C032
:103C3000511139C1F3C014D198F39923C9F3552315
:103C4000B1F3951B550BBB27AA276217730784078F
:103C500038F09F5F5F4F220F331F441FAA1FA9F345
:103C600033D00E2E3AF0E0E830D091505040E69537
:103C7000001CCAF729D0FE2F27D0660F771F881F98
:103C8000BB1F261737074807AB07B0E809F0BB0B87
:103C9000802DBF01FF2793585F4F2AF09E3F5105AB
:103CA00068F0B6C000C15F3FECF3983EDCF3869548
:103CB00077956795B795F7959F5FC9F7880F911D21
:103CC0009695879597F90895E1E0660F771F881F0D
:103CD000BB1F621773078407BA0720F0621B730BC0
:103CE000840BBA0BEE1F88F7E095089504D0689412
:103CF000B111D9C00895BCD088F09F5790F0B92F6A
:103D00009927B751A0F0D1F0660F771F881F991F30
:103D10001AF0BA95C9F712C0B13081F0C3D0B1E042
:103D20000895C0C0672F782F8827B85F39F0B93F52
:103D3000CCF3869577956795B395D9F73EF4909532
:103D40008095709561957F4F8F4F9F4F0895E894B0
:103D500009C097FB3EF490958095709561957F4FD3
:103D60008F4F9F4F9923A9F0F92F96E9BB27939581
:103D7000F695879577956795B795F111F8CFFAF491
:103D8000BB0F11F460FF1BC06F5F7F4F8F4F9F4FC2
:103D900016C0882311F096E911C0772321F09EE820
:103DA000872F762F05C0662371F096E8862F70E086
:103DB00060E02AF09A95660F771F881FDAF7880F60
:103DC0009695879597F90895990F0008550FAA0BB6
:103DD000E0E8FEEF16161706E807F907C0F012161E
:103DE0001306E407F50798F0621B730B840B950B21
:103DF00039F40A2661F0232B242B252B21F4089576
:103E00000A2609F4A140A6958FEF811D811D089512
:103E100097F99F6780E870E060E008959FEF80EC7D
:103E2000089500240A941616170618060906089520
:103E300000240A9412161306140605060895092E86
:103E40000394000C11F4882352F0BB0F40F4BF2BF5
:103E500011F460FF04C06F5F7F4F8F4F9F4F089535
:103E600057FD9058440F551F59F05F3F71F047952B
:103E7000880F97FB991F61F09F3F79F08795089510
:103E8000121613061406551FF2CF4695F1DF08C02F
:103E9000161617061806991FF1CF8695710561054C
:103EA00008940895E894BB2766277727CB0197F9F4
:103EB00008958ADF08F48FEF08950BD0C0CFB1DFEB
:103EC00028F0B6DF18F0952309F0A2CFA7CF112470
:103ED000EACFC6DFA0F3959FD1F3950F50E0551FB1
:103EE000629FF001729FBB27F00DB11D639FAA274F
:103EF000F00DB11DAA1F649F6627B00DA11D661F9E
:103F0000829F2227B00DA11D621F739FB00DA11DBE
:103F1000621F839FA00D611D221F749F3327A00D78
:103F2000611D231F849F600D211D822F762F6A2F14
:103F300011249F5750408AF0E1F088234AF0EE0F99
:103F4000FF1FBB1F661F771F881F91505040A9F7A6
:103F50009E3F510570F05CCFA6CF5F3FECF3983EDB
:103F6000DCF3869577956795B795F795E7959F5F0D
:103F7000C1F7FE2B880F911D9695879597F90895A7
:103F8000FA01EE0FFF1F30962105310599F16115F9
:103F9000710561F48038BFE39B0749F1689490385C
:103FA000810561F08038BFEF9B0741F0992342F50E
:103FB000FF3FE1053105210511F1E8940894E795EB
:103FC000D901AA2329F4AB2FBE2FF85FD0F310C07C
:103FD000FF5F70F4A695E0F7F73950F019F0FF3A5B
:103FE00038F49F779F930CD00F9007FC905808955A
:103FF0003EF014CF60E070E080E89FE308954FE763
:104000009F775F934F933F932F939ED02F913F9134
:104010004F915F9152DF05C019F40EF0F9CE42CFF7
:10402000FDCE26DFC8F39638C0F707F80F92E89464
:104030002BE33AEA48EB5FE74EDF0F920F920F92C5
:104040004DB75EB70F92C0D0E8EEF0E016D04F91BA
:104050005F91EF91FF91E595EE1FFF1F49F0FE572D
:10406000E0684427EE0F441FFA95E1F74195550BA0
:1040700032D00F9007FE26C00895DF93CF931F9391
:104080000F93FF92EF92DF927B018C01689405C041
:10409000DA2EEF011EDFFE01E894A59125913591FE
:1040A00045915591AEF3EF0162DDFE019701A80144
:1040B000DA9479F7DF90EF90FF900F911F91CF91F5
:1040C000DF9108959B01AC0160E070E080E89FE320
:1040D000A5CD9ECEACC0CCDEE8F39923D9F3940FE6
:1040E000511DBBF39150504094F059F0882332F0A9
:1040F000660F771F881F91505040C1F79E3F5105B2
:1041000044F7880F911D9695879597F908955F3F1D
:10411000ACF0983E9CF0BB27869577956795B79550
:1041200008F4B1609395C1F7BB0F58F711F460FF25
:10413000E8CF6F5F7F4F8F4F9F4FE3CFB4CE0EF02E
:1041400076C06CCE689464CE93DEC8F39923D1F325
:10415000C6F3DF93CF931F930F93FF92C92FDD27F1
:1041600088232AF02197660F771F881FDAF720E04F
:1041700030E040E85FEB9FE3883920F0803E30F08C
:1041800021968F77E3DCE0E1F1E003C0DFDCEDE3D3
:10419000F1E073DF8B01BE01EC01FB2E6F5771095B
:1041A0007595771F880B990BD4DD28E132E741E341
:1041B0005FE38FDEAF2D9801AE01FF900F911F914D
:1041C000CF91DF91D4DC3BCEFA01DC01AA0FBB1FFB
:1041D0009B01AC01BF5728F422273327442750788E
:1041E0001FC0B75188F4AB2F00244695379527950B
:1041F000011CA395D2F3002069F0220F331F441F46
:10420000B395DAF30DD0A1CC61307105A0E88A072F
:10421000B94630F49B01AC01662777278827907850
:10422000309621F0208331834283538308959F3F4A
:1042300031F0915020F4879577956795B795880F61
:10424000911D9695879597F90895DB018F939F931C
:104250000E946121BF91AF91A29F800D911DA39FEC
:10426000900DB29F900D11240895052E97FB1EF41A
:1042700000940E944C2157FD07D00E94742107FC36
:1042800003D04EF40C944C215095409530952195D7
:104290003F4F4F4F5F4F0895909580957095619572
:1042A0007F4F8F4F9F4F0895EE0FFF1F0590F491A2
:1042B000E02D09940E949621B7FF0895821B930B6D
:1042C00008950E949621A59F900DB49F900DA49FE4
:1042D000800D911D11240895B7FF0C9461210E9457
:1042E0006121821B930B0895A1E21A2EAA1BBB1B0E
:1042F000FD010DC0AA1FBB1FEE1FFF1FA217B307B2
:10430000E407F50720F0A21BB30BE40BF50B661FC7
:10431000771F881F991F1A9469F76095709580958B
:1043200090959B01AC01BD01CF010895A29FB00102
:10433000B39FC001A39F700D811D1124911DB29FD9
:0E434000700D811D1124911D0895F894FFCF7A
:10434E000000D70280000100002AD432B2122514D8
:10435E0002E1C5025F5A050F26FCA5A5D6DDDCFCE1
:10436E00252B22210FFFF8EEEDEFF7F6FA000302F0
:10437E0001CDDFF10416203B4DC0D4E8FC102539E9
:10438E004DC0D8F0071F374F66B3BFCBD7E3EFFB57
:10439E0007131F2B37434F5A66C0CBD6E1ECF703FA
:1043AE000E19242F3A45505B66AEBAC5D1DDE8F43E
:1043BE00FF0B17222E3945515CAEBCCAD8E6F4016C
:1043CE000F1D2B39475563717E929FADBAC8D5E349
:1043DE00F0FE0B192634414F5CAEB5BCC3CCD4DE17
:1043EE00E8F2FC06101A242D363E464D53595E62F5
:1043FE00666A6D70727476777F8384848485858611
:10440E0088898A8B8C8D8F919399A1ACB8C7D9EC82
:10441E000014273948555F676D00101112131415DB
:10442E00161718191A1B1C1D1E1F202122232425A6
:10443E00262728292A2B2D2F31333536393B3D3F60
:10444E00424547494D4F5155575C5F63666A6E73DF
:10445E00777B80858A8F959AA00002030405070A50
:10446E000F142029395172A1FF0E0F1011121300D3
:10447E00010108000A0A0A0A0A0A0A0A01015B1B5C
:02448E005B1BB6
:00000001FF
